:1000000041230D3084007C280B1D09009000030E55
:100010008F008312851D0E2891011328110F910066
:100020004120FF309C00051E172892011C28120F4A
:1000300092004120FF309C00061C202893012328B9
:10004000130F930041201A081B0403192C289B0F3F
:100050002C289A0F2C289D151708031D9703180AA2
:10006000031935281808031D98031C0803193B2899
:100070009C0B3B281D160F0E8300900E100E0B11CB
:100080000900FB309A00B4309B000800820754340A
:1000900058340034523458340034583400344C341A
:1000A0000034203400342034443449345334503440
:1000B0004C3441345934203400344D3455344C34AC
:1000C000543400344D344134583400344D344934C0
:1000D0004E34203400342034563443344F342034EA
:1000E0004F34463446345334453454342034003489
:1000F0004D3448347A34003443308C008001840A13
:100100008C0B7E288316183085000330860004305F
:10011000810083128101A0308B00FE30860086149E
:10012000FE21061C9D16652341209D119030D6218D
:100130000830DC216B219D1994287123051DA4280A
:100140001D1F9D171D17A7281D1B9D171D138F30E1
:10015000D62106301D1DAF281F1FAF280A30DC2115
:100160009D1FB5289C1BCD289D131D1FC228243020
:100170002C23492328303A2325232A303A231823D5
:100180002430CC2826302C2349232E303A23252313
:1001900030303A23182326303323B5217D219D1E8C
:1001A0009B28CE23191C9B28D0210C30DC21163033
:1001B000DC219D199428B5219F231918A30AB02387
:1001C0001918A303013023020318E8280130A30003
:1001D00015302302031CEE281430A300C2012308AB
:1001E000C3000A304302031CF828C300C20AF128E6
:1001F0008E30D6214208303ECC214308303ECC21FF
:100200009623191CD928D5211F30DC210330DC218D
:100210000C30DC216B219D199428B52128307221E6
:10022000283033237D219623191C0B29D5211B301F
:10023000DC219D199428B5212A302C23492328300C
:1002400070212A3033237D219623191C1929D521A9
:100250000330DC212430DC219D199428B5212C3079
:10026000A4212C3033237D219623191C2C29D52140
:100270001F30DC210030DC210C30DC219D1994285A
:10028000B5212E3072212E3033237D219623191C67
:100290003E29D5211B30DC219D199428B521303011
:1002A0002C2349232E307021303033237D21962397
:1002B000191C4C29D5210030DC212430DC219D196A
:1002C0009428B5213230A421323033237D21962366
:1002D000191C5F2994288A30D6213130DC2108008E
:1002E0003A2376292C234923B901BA012523553015
:1002F000B900F030BA00182308009D103709C03942
:10030000031D89299D14B709B8090130B8070318DE
:10031000B70A2308B6000310B70D0310B80D031871
:10032000B70A0310E12289228030D62141308400AF
:1003300008308C000008CC21840A8C0B9A29883064
:10034000D6210008CC2108002C238030B706492391
:100350008130B9009030BA0018237E30B900703077
:10036000BA0025238030B70608003822051DBE29B3
:1003700024302C23213033232C30C32926302C2346
:100380002130332332303A230123142221302C230D
:100390000800CB21CB212030A100A2008615E52941
:1003A0000130D6211830422308008130A100A2007C
:1003B0008611E52186150800A0004620FF390319A3
:1003C0000800CC212008013EDC29051183160130EC
:1003D000860083120615F030A10506080E392104A7
:1003E000860006110615A20EF030A20506080E3989
:1003F0002204860006114B308522080086010F2258
:100400000F220F2228308600061141232830D621E2
:100410000830D621D0210630D6210C30D6294123F0
:1004200038308600061108009E101D155E230F301F
:10043000B900A030BA0025235430B9006030BA00AA
:10044000182334303A230F230319352A3430332349
:100450006A22C2305C2237085C2238085C228E3067
:100460005C2200305C226F221F139E181D110800B1
:100470001F1F3E2A1808031D502A59226A22C33022
:100480005C2208308C00842205148422060C9F0D07
:1004900005108C0B432A802276226F221F1B5922C3
:1004A000051D1F1F572A1D1D572A86100800861478
:1004B00008006E3098000800A00008308C00A00DE5
:1004C00003188022031C7B2276228C0B5F2A802259
:1004D000762208000514802284227B22782A7B223F
:1004E0008422051484228022842208008422051498
:1004F00084220510080085108316851083120800D9
:1005000083168514831208000F308D008D0B862A08
:100510000800031018308C00C201C401C701C901D2
:10052000BF0DBE0DBD0DC90DC70DC40DC20D8C0B89
:10053000BC2A490EC800470EC500440EC300420E37
:10054000C1001D104130D1224230D1224330D1228E
:100550004430D1224530D1221D144730D122A5305C
:10056000C6004830D1224930D1229D1C08004008E5
:1005700084002D30800008004930C5224730C52254
:100580004430C5224230C522902A8400033000073F
:10059000A000A019800030300007A000A01B800040
:1005A000080084000F3000050319DA2A303E80006D
:1005B0001D1408001D18D62A203080000408C00031
:1005C0000800BF013708BD003808BE0008308C00A5
:1005D000B60C0318F02A8C0BE82ABD01BE010800F6
:1005E0000310FB2AB60C031CFB2A3808BE07370889
:1005F0000318370FBD07BD0CBE0CBF0C8C0BF22AC5
:1006000008003A08B80739080318390FB707080077
:100610003A08B8023908031C390FB70208003A0833
:100620003802A0003908031C390A370220040800E8
:100630003908BB003A08BC000130BA070318B90AF0
:100640000F23031C08003B30292B0F23031808003D
:1006500039302C239E14080084000008B700840A57
:100660000008B8000800840037088000840A3808B1
:100670008000080084000008B900840A0008BA005D
:10068000080076308D008E018E0B442B8D0B442B91
:100690000800B9010130061C1430BA00A72319184C
:1006A0000123B823191808230230061CC830BA00E9
:1006B0009F2319180123B023191808233709C039BB
:1006C000031D0800B701B801080089012330840028
:1006D00011308C0084238000890A840A8C0B6A2BD9
:1006E00008001D1E08001D128901233084001130EE
:1006F0008C008423000203197F2B00088923890AB8
:10070000840A8C0B792B08008316081483120808BE
:100710000800880083160812081555308900AA3091
:1007200089008814081E922B831208001E30A00036
:10073000160899001302C1231308960008006430BC
:100740001102031CA72B463091006630A82B3C30C9
:10075000A000140899001102C12311089400080098
:1007600064301202031CB82B463092006630B92B5D
:100770003C30A000150899001202C1231208950010
:1007800008000318CB2B1908053C0318CB2B1908BC
:100790002002FF30031C0301990008009623191C56
:1007A000080017080319D52B080019309700CB2B28
:02400E00FA3F77
:10420000FA004F00A400510038004E002000520078
:104210000800000000004E002000520008000000CE
:0242200000009C
:00000001FF
